:03000000020100FA
:0300230002028B4B
:1001000031CA51A1758920758DFD75985075A890DB
:10011000D28E51A175A000790020B00451AE80F9B3
:10012000B9391275900F517C51819001F5513B51B5
:10013000AE31CA80E4B9321275A00A517C51819067
:1001400001FF513B51AE31CA80CFB9331275A005C2
:10015000517C5181900207513B51AE31CA80BAB9EE
:10016000341275A009517C5181900210513B51AE5F
:1001700031CA80A5B9351275A006517C5181900213
:1001800015513B51AE31CA8090B9361275A0085155
:100190007C518190021B513B51AE31CA2119B937B4
:1001A0001275A002517C5181900228513B51AE3111
:1001B000CA2119B9381275A000517C5181900236BC
:1001C000513B51AE31CA21192119517C5145518100
:1001D0009001DD513B51869001ED513B2220564F5D
:1001E00049434520434F4E54524F4C200020524F1C
:1001F000424F542000434F4E4E4543544544004621
:100200004F5257415244004241434B5741524400E0
:100210004C454654005249474854005245564552B1
:100220005345204C454654005245564552534520AF
:1002300052494748540053544F5000E493600551CD
:100240006BA380F7227430515A7438515A74065196
:100250005A740C515A7401515A2251AE51AEC29582
:10026000C296D297F5800000C2972251AE51AED20D
:1002700095C296D297F5800000C297227401515A18
:10028000227480515A2274C0515A22209803209916
:0A0290000BC298E599F951B7D2B0FE
:10029A008004C2998000227B107CC87DFADDFEDCD6
:1002AA00FADBF6227BB77CFADCFEDBFA227B287CBF
:0602BA00FADCFEDBFA2273
:00000001FF
